:10000000B401962AB521B6000408B8000800B5214D
:10001000B7000408B9000800B600AE2184133230DE
:10002000A600A7017022A00AA50AA201A301000848
:100030003605A600640000083605A7002606270539
:1000400036060319A20A0319A30A2708A600A40367
:100050000319A5030319A00B1A282208912A0408E2
:10006000A2008316861183120930A30003103F20DB
:10007000A20CA30B372803143F200314912A031862
:100080004428000086154628861146280030A10025
:10009000C330002A0408A7000610861086108316B5
:1000A0000610861086100F30860583122708B418B4
:1000B00077283A30A100983000223330A6008B20F8
:1000C0001330A100883000228B206430FF218B2068
:1000D0006430FF212230A6008B20283076200C309F
:1000E000762006307620B414270877283414A6002A
:1000F000341C85288610033C031C8A288A2007307C
:10010000A100D0300022031408003414FE3C03196F
:10011000912A8614341C341006140F3086052608E4
:10012000F03986040610A60E34188B283230FF21D1
:1001300003140800B521B600B121200821040319D9
:10014000912A86228413360880066400A728A828EE
:10015000A00A0319A10FA5288006912A6400C420D3
:100160000318AE281121A8010830A3001221C420D1
:100170000318A80AAB1EA801A20CA30BB628AB1A41
:10018000A2131221220808003808840036088417B8
:100190008004841300052B1B3606FF3E0800290847
:1001A0000319912A8C22A903CF28A401A501B51215
:1001B0008C22D33E0319B5162D3EC63E0318E42803
:1001C0000A3E031CD828EB28F33E0318D828063E25
:1001D000031CD8280A3EA2000430A3000310A40D7B
:1001E000A50DA30BEE282208A404A90303190829CE
:1001F0008C22C63E031800290A3E031C0829EB285E
:10020000F33E03180829063E031C08290A3EEB2882
:10021000B51E0F29A409A509A40A0319A50A2408D3
:10022000912A35172B081F39FF3EA1002A08F53EF9
:100230000318A10A351F002A3513A000023032220C
:10024000002AB51329080319B5170430A800250E94
:100250002E2125082E21240E2E2124080F39F63EAA
:100260000318073E0A3E5129B51329080319B5178B
:100270000530A8002730A30010304A210330A30026
:10028000E8304A21A30164304A21A3010A304A21FF
:1002900024085129A2002508A1002408A000542206
:1002A0002008A000A8030319B513290803195B2926
:1002B0002802031808002008031DB513B51B080009
:1002C000303E8C2A0830A600A70039088400370881
:1002D00035198004FF3A351D8005B22138088400A5
:1002E0003608AE21A001A101B518A221380884006A
:1002F00000083605FF3EA00DA10DB51CA221A60BDE
:10030000742927083518142A2008912A0830A600D5
:10031000351814223908840037083519A921351DEC
:10032000AB21380884003609B22138088400A10CBA
:10033000A00C00083604031C36068000A221A60B80
:100340009529912A39088400370880060000800624
:1003500008008004B129FF3A8005B229841780047F
:10036000912AFF3A84178005912AA8000630A8191F
:100370000730840001308A002808073982070134D9
:100380000234043408341034203440348034A00063
:10039000A00DA00DA00D3830A005813020049F00D5
:1003A0000030A100323000221F151F19D5291E0868
:1003B000A10083161E08912A03178D0083168C1343
:1003C0000C1483120C08912A03178C0083168C13CB
:1003D0000C1555308D00AA308D008C148C18EE2928
:1003E0000C11912AA301A200FF30A207031CA3074E
:1003F000031C912A0330A100DF300022F429A1015F
:10040000E83EA000A109FC30031C092AA00703183C
:10041000062AA0076400A10F062A20180F2AA01C94
:10042000132A0000132A0800A400A201A3011C2A19
:10043000A10CA00CA20DA30DFF3E0318182A24083E
:100440002A222208A0042308A1042008080003107F
:10045000A00DA10DFF3E0318272A2008912A0310A2
:10046000A10CA00CFF3E03182F2A2008912AA200FD
:100470000330442AA301A2000130442AA20006301E
:10048000442AA2000430442AA80023082102031DA4
:100490004B2A2208200204300318013003190230CD
:1004A0002805031DFF30912A1030A600A501A401E4
:1004B000210DA40DA50D2208A4022308031C230F5F
:1004C000A50203186A2A2208A40723080318230F89
:1004D000A5070310A00DA10DA60B582A2008912AEC
:1004E0001030A800A101A001A70CA60C031C7E2AB5
:1004F0002208A00723080318230FA107A10CA00CB2
:10050000A50CA40CA80B742A2408912AA009A109FF
:10051000A00A0319A10A0800840031088A003008E3
:100520008200831303138312640008000330A300C6
:10053000E8308A01F3218316043086001F308500DD
:10054000FC3087008312831684309F008312813031
:100550009F0064008A110A12071EB52A64008A11DE
:100560000A12071A722F8A01A92AFE308A014B202B
:1005700001308A014B2043308A014B2061308A01CF
:100580004B206C308A014B2069308A014B2062304D
:100590008A014B2072308A014B2061308A014B2046
:1005A00063308A014B2069308A014B206F308A0109
:1005B0004B206E308A014B2043308A01302061305D
:1005C0008A0130206C308A01302069308A01302065
:1005D00062308A01302072308A01302061308A0115
:1005E000302063308A01302069308A0130206F303A
:1005F0008A0130206E308A01302020308A0130207C
:100600002D308A01302020308A01302065308A0167
:1006100030206E308A01302074308A0130207230F0
:100620008A01302061308A01302072308A01302006
:1006300020308A01302076308A01302061308A01F2
:1006400030206C308A0130206F308A0130207230C7
:100650008A01302065308A01302073308A013020D1
:100660000A308A0130200D308A01302043308A015F
:1006700030206F308A0130206D308A013020703098
:100680008A01302065308A0130206E308A013020A6
:1006900073308A01302061308A01302063308A0152
:1006A000302069308A0130206F308A0130206E306E
:1006B0008A01302020308A01302054308A013020D5
:1006C00065308A0130206D308A01302070308A0117
:1006D00030202B308A0130203A308A0130200A3015
:1006E0008A0130200D308A0130200530B8002030DA
:1006F000B600BC30AA004030AB000130A900AE30DB
:10070000B000B1018A01D520FD000130A9007D08AB
:10071000A400A5012F30B000B1018A0121210A30C7
:100720008A0130200D308A013020FE308A014B20B2
:10073000C0308A014B2054308A014B2065308A0139
:100740004B206D308A014B2070308A014B202030C5
:100750008A014B202B308A014B200130A9007D08F3
:10076000A400A5014A30B000B1018A01212103177C
:1007700001308D0003137D088A01E4210330A300BA
:10078000E8308A01F321FE308A014B2001308A01D2
:100790004B2043308A014B2061308A014B206C3062
:1007A0008A014B2069308A014B2062308A014B203C
:1007B00072308A014B2061308A014B2063308A01FC
:1007C0004B2069308A014B206F308A014B206E30FC
:1007D0008A014B2043308A0130206F308A0130205B
:1007E0006D308A01302070308A01302065308A01F6
:1007F00030206E308A01302073308A013020613021
:100800008A01302063308A01302069308A0130202B
:100810006F308A0130206E308A01302020308A010A
:10082000302054308A01302065308A0130206D300C
:100830008A01302070308A0130202D308A0130202A
:100840003A308A0130200A308A0130200D308A0186
:1008500030200530B8002030B600BC30AA0040304F
:10086000AB000130A900AE30B000B1018A01D52043
:10087000FD000130A9007D08A400A5012F30B000C3
:10088000B1018A0121210A308A0130200D308A010C
:100890003020FE308A014B20C0308A014B2054307A
:1008A0008A014B2065308A014B206D308A014B2034
:1008B00070308A014B2020308A014B202D308A0174
:1008C0004B200130A9007D08A400A5014A30B000EA
:1008D000B1018A012121031702308D0003137D0825
:1008E0008A01E4210330A300E8308A01F321FE30BD
:1008F0008A014B2001308A014B2043308A014B2072
:1009000061308A014B206C308A014B2069308A01AA
:100910004B2062308A014B2072308A014B206130BB
:100920008A014B2063308A014B2069308A014B20B9
:100930006F308A014B206E308A014B2043308A0190
:1009400030206F308A0130206D308A0130207030C5
:100950008A01302065308A0130206E308A013020D3
:1009600073308A01302061308A01302063308A017F
:10097000302069308A0130206F308A0130206E309B
:100980008A01302020308A01302048308A0130200E
:1009900075308A0130206D308A0130202B308A0179
:1009A00030203A308A0130200A308A0130200D3060
:1009B0008A0130200530B8002030B600BC30AA00D3
:1009C0004030AB000130A900AE30B000B1018A0167
:1009D000D520FD000130A9007D08A400A5012F301D
:1009E000B000B1018A0121210A308A0130200D3086
:1009F0008A013020FE308A014B20C0308A014B2012
:100A000048308A014B2075308A014B206D308A01B5
:100A10004B2020308A014B202B308A014B200130A3
:100A2000A9007D08A400A5014A30B000B1018A01E7
:100A30002121031703308D0003137D088A01E4216F
:100A40000330A300E8308A01F321FE308A014B20F5
:100A500001308A014B2043308A014B2061308A01EA
:100A60004B206C308A014B2069308A014B20623068
:100A70008A014B2072308A014B2061308A014B2061
:100A800063308A014B2069308A014B206F308A0124
:100A90004B206E308A014B2043308A0130206F306A
:100AA0008A0130206D308A01302070308A01302078
:100AB00065308A0130206E308A01302073308A011F
:100AC000302061308A01302063308A013020693063
:100AD0008A0130206F308A0130206E308A01302048
:100AE00020308A01302048308A01302075308A0158
:100AF00030206D308A0130202D308A0130203A308C
:100B00008A0130200A308A0130200D308A013020DD
:100B10000530B8002030B600BC30AA004030AB0031
:100B20000130A900AE30B000B1018A01D520FD002E
:100B30000130A9007D08A400A5012F30B000B1014B
:100B40008A0121210A308A0130200D308A013020AB
:100B5000FE308A014B20C0308A014B2048308A0188
:100B60004B2075308A014B206D308A014B2020309C
:100B70008A014B202D308A014B200130A9007D08CD
:100B8000A400A5014A30B000B1018A012121031758
:100B900004308D0003137D088A01E4210330A30093
:100BA000E8308A01F321FE308A014B2001308A01AE
:100BB0004B2043308A014B2061308A014B206C303E
:100BC0008A014B2069308A014B2062308A014B2018
:100BD00072308A014B2061308A014B2063308A01D8
:100BE0004B2069308A014B206F308A014B206E30D8
:100BF0008A014B2043308A0130206F308A01302037
:100C00006D308A01302070308A01302065308A01D1
:100C100030206E308A01302073308A0130206130FC
:100C20008A01302063308A01302069308A01302007
:100C30006F308A0130206E308A01302020308A01E6
:100C4000302050308A01302072308A0130206530E7
:100C50008A01302073308A01302073308A013020BD
:100C60002B308A0130203A308A0130200A308A0144
:100C700030200D308A0130200530B8002030B60019
:100C8000BC30AA004030AB000130A900AE30B0004B
:100C9000B1018A01D520FD000130A9007D08A40022
:100CA000A5012F30B000B1018A0121210A308A014B
:100CB00030200D308A013020FE308A014B20C030B8
:100CC0008A014B2050308A014B2072308A014B2020
:100CD00065308A014B2073308A014B2073308A01C2
:100CE0004B2020308A014B202B308A014B200130D1
:100CF000A9007D08A400A5014A30B000B1018A0115
:100D00002121031705308D0003137D088A01E4219A
:100D10000330A300E8308A01F321FE308A014B2022
:100D200001308A014B2043308A014B2061308A0117
:100D30004B206C308A014B2069308A014B20623095
:100D40008A014B2072308A014B2061308A014B208E
:100D500063308A014B2069308A014B206F308A0151
:100D60004B206E308A014B2043308A0130206F3097
:100D70008A0130206D308A01302070308A013020A5
:100D800065308A0130206E308A01302073308A014C
:100D9000302061308A01302063308A013020693090
:100DA0008A0130206F308A0130206E308A01302075
:100DB00020308A01302050308A01302072308A0180
:100DC000302065308A01302073308A013020733042
:100DD0008A0130202D308A0130203A308A013020BB
:100DE0000A308A0130200D308A0130200530B800E9
:100DF0002030B600BC30AA004030AB000130A90062
:100E0000AE30B000B1018A01D520FD000130A9004B
:100E10007D08A400A5012F30B000B1018A01212175
:100E20000A308A0130200D308A013020FE308A01DC
:100E30004B20C0308A014B2050308A014B20723049
:100E40008A014B2065308A014B2073308A014B2088
:100E500073308A014B2020308A014B202D308A01CB
:100E60004B200130A9007D08A400A5014A30B00044
:100E7000B1018A012121031706308D0003137D087B
:100E80008A01E4210330A300E8308A01F321FE3017
:100E90008A014B2001308A014B2050308A014B20BF
:100EA00075308A014B206C308A014B2073308A01E7
:100EB0004B2061308A014B2072308A014B20203058
:100EC0008A014B2052308A014B2065308A014B2029
:100ED00073308A014B2065308A014B2074308A01BF
:100EE0004B200800FE308A014B2001308A014B2044
:100EF00020308A014B2050308A014B2049308A0132
:100F00004B2043308A014B202D308A014B20573033
:100F10008A014B2058308A014B2020308A014B2017
:100F200053308A014B2054308A014B2041308A01D2
:100F30004B2054308A014B2049308A014B204F30DE
:100F40008A014B204E308A014B2020308A014B20F1
:100F5000FE308A014B20C0308A014B2045308A0187
:100F60004B2041308A014B2033308A014B204330E3
:100F70008A014B204E308A014B204F308A014B2092
:100F800020308A014B2020308A014B2057308A01C3
:100F90004B2058308A014B205F308A014B20413072
:100FA0008A014B2050308A014B2052308A014B205D
:100FB00053308A014B2043308A014B200B30A30071
:100FC000B8308A01F3218716831687120F308312F7
:100FD0008A0102200E308A010720B5010C30A000E2
:100FE000A1018A0186210230A000A1018A01862187
:100FF0008712831687128312F901F501F601C201E7
:10100000C3018316A601831200308A01C721C000E4
:101010002108C10001308A01C721BA002108BB00A4
:10102000CA30A2000830A3000630840004308A01D0
:101030000C208316A70005308312B8000430B600D8
:10104000BC30AA004030AB008A01AE202A3C8A1591
:101050000A12031D24280230A900AE30B000B101ED
:101060008A01D520F7000130A900AE30B000B101EF
:101070008A01CF200230A900AE30B000B1018A0150
:10108000D520FA000130A900AE30B000B1018A01CC
:10109000CF200230A900AE30B000B1018A01D520C6
:1010A0008316A00083120130A900AE30B000B10158
:1010B0008A01CF200230A900AE30B000B1018A0110
:1010C000D520F2000130A900AE30B000B1018A0194
:1010D000CF200230A900AE30B000B1018A01D52086
:1010E000FB000130A900AE30B000B1018A01CF2071
:1010F0000230A900AE30B000B1018A01D5208316BC
:10110000A800013083128A01DC21F10002308A013B
:10111000DC21F00003308A01DC21ED0004308A017B
:10112000DC21EC0005308A01DC21EF0006308A0169
:10113000DC21EE008A150A12D9218A150A120F2223
:101140007108D0070318D10A7008D002031CD1031C
:101150008A150A1236228A150A1265228A150A127F
:1011600094228A150A12F1228A150A126F238A150F
:101170000A128D238A150A129D238A150A12E12369
:101180008A150A120A2464008A150A12871D8B2DFB
:1011900064008A150A12071EFF2D5008A00051088E
:1011A000A1000130A30000308A0137228A150A12FB
:1011B000031D7B2C5008A0005108A1000130A300A2
:1011C00000308A0141228A150A12031D032D8A1557
:1011D0000A124E248A150A125D248A150A126C24FA
:1011E000C20A0319C30A4208A0004308A100A301D0
:1011F00004308A013E228A150A12031D0428033096
:10120000A9003E08A4003F08A5002F30B000B1019E
:101210008A0134212C308A0130200330A9004A0889
:10122000A4004B08A5002F30B000B1018A01342181
:101230002C308A0130200330A9007508A400A501D4
:101240002F30B000B1018A0134212C308A013020C6
:101250000330A9005008A4005108A5002F30B000A9
:10126000B1018A0134212C308A0130200430A900D8
:101270004408A4004508A5002F30B000B1018A0140
:1012800034212C308A0130200230A9007808A400D3
:10129000A5012F30B000B1018A0134212C308A0120
:1012A00030200230A9007208A400A5012F30B00040
:1012B000B1018A0121212C308A0130200230A9009D
:1012C0007708A400A5012F30B000B1018A012121C7
:1012D0002C308A0130200230A9007A08A400A50130
:1012E0002F30B000B1018A0121212A308A0130203B
:1012F0000330A9004C08A4004D08A5002F30B00011
:10130000B1018A0134212C308A0130200330A90038
:101310007608A400A5012F30B000B1018A01342164
:101320002C308A0130200330A9008316250883124F
:10133000A400A5012F30B000B1018A0134212A3068
:101340008A0130202A308A0130200230A900831619
:1013500021088312A400A5012F30B000B1018A0139
:1013600034212E308A013020A901831623088312EC
:10137000A400A5012F30B000B1018A0134210A3048
:101380008A0130200D308A013020C201C30183164A
:10139000A60A64002D3026028A150A128312031C45
:1013A0000428F501F6018316A60183128A150A1294
:1013B00004288716831687120F3083128A010220B1
:1013C0000E308A010720B501EE30A000A1018A018C
:1013D0008621871283168712831287168316871237
:1013E0000F3083128A0102200E308A010720B501D6
:1013F000AA30A000A1018A0186210F308A010220B3
:101400000E308A0107200130B5008A016221CE002A
:101410002108CF00871283168712831208004E0816
:10142000A0004F08A100A301C8308A0141228A15FB
:101430000A12031D282A4E08A0004F08A100A3018C
:10144000C9308A0137228A150A12031D312A080081
:1014500000304E07D00001300318013E4F07D10085
:1014600008004E08D0004F08D1000800003050029C
:10147000B2000130031C013E5102B300330C320CA8
:101480008316A100003083125002B2000130031C09
:10149000013E5102B3003208A0003308A10002301F
:1014A000A200A3018A0154222408B2002508B30037
:1014B0003208A6003308A7000530A200A3018A0164
:1014C00070228316A300831208005008003CB2006B
:1014D0005108031C013E013CB300330C320C83164F
:1014E000A20083125008003CB2005108031C013EC8
:1014F000013CB3003208A0003308A1000230A20072
:10150000A3018A0154222408B2002508B30032083E
:10151000A6003308A7000530A200A3018A017022AB
:101520008316A40083120800510C500CF3005008DD
:10153000A0005108A1000230A200A3018A01542298
:101540002408B2002508B3003208A6003308A7001B
:101550000530A200A3018A017022F40092307307C3
:10156000B200FF300318013EB3003208A600330872
:10157000A7000A30A200A3018A017022BC0025083E
:10158000BD003C08A0003D08A1000530A200A30159
:101590008A015422B2002108B3003208A6003308A1
:1015A000A7000930A200A3018A017022B200250819
:1015B000B3003208A0003308A1000A30A200A30142
:1015C0008A0154228316A500640005308312740238
:1015D0008A150A120318ED2A08008316A50A831239
:1015E00008003A08A6003B08A7003230A200A30179
:1015F0008A017022B2002508B3003208A000330827
:10160000A100FF30A2000330A3008A015422C600CB
:101610002108C7003A08A6003B08A7003230A20004
:10162000A3018A017022B2002508B3003208A0008D
:101630003308A100FF30A2000330A3008A01542226
:101640002408C8002508C9004608A6004708A700C6
:10165000E830A2000330A3008A017022B2002508FE
:10166000B3004808B20749080318013EB30732081F
:10167000A0003308A100F430A2000130A3008A01C9
:101680005422B2002108B3001030B2020030031C13
:10169000013EB3023208A6003308A7006430A2005E
:1016A000A3018A017022B2002508B3003208A0000D
:1016B0003308A1003E30A200A3018A015422F800A1
:1016C0006D08F8076C08F8026400643078028A1527
:1016D0000A1203186C2B08006330F800080007108A
:1016E00083160710831287108316871083126430C5
:1016F000A000A10109308A019A200A308A01022043
:1017000009308A0107200230B5008A016221FC00FD
:101710000714831607108312080020307C07C400CA
:1017200003300318013EC5006F08C4070318C50A3B
:101730006E08C402031CC503080083162708831221
:10174000A600A701A330A200A3018A017022B20063
:101750002508B3003208A0003308A1006430A200BD
:10176000A3018A015422B2002108B30001303202E1
:10177000CA000030031C013E3302CB008316270849
:101780008312A600A701A330A200A3018A01702240
:10179000B2002508B3003208A0003308A10064306D
:1017A000A200A3018A0154222408FE006400343000
:1017B0007E028A150A120318DD2BCA0A0319CB0A06
:1017C00008002430A600A7014008A2004108A30099
:1017D0008A017022B2002508B3003208A000330845
:1017E000A1006630A200A3018A015422BE00210894
:1017F000BF003E08A0003F08A1000130A3006830F0
:101800008A0137228A150A12031D072C0800BE011F
:10181000BF010800831627088312A600A7016730BE
:10182000A200A3018A017022B2002508B300320889
:10183000A0003308A1006430A200A3018A01542251
:10184000B2002108B30001303202CC000030031C8A
:10185000013E3302CD00831627088312A600A7019C
:101860006730A200A3018A017022B2002508B300EC
:101870003208A0003308A1006430A200A3018A014D
:1018800054222408FF00640034307F028A150A12B3
:1018900003184A2CCC0A0319CD0A08004A08A000F4
:1018A0004B08A10079088A013A228A150A12031D01
:1018B0005A2C08004A08F90008004A08A0004B0802
:1018C000A10075088A013A228A150A12031D692CA3
:1018D00008004A08F50008004C08A0004D08A100C7
:1018E00076088A013A228A150A12031D782C08000C
:1018F0004C08F6000800FE308A014B2001308A01B6
:101900004B202B308A014B200230A900831621087E
:101910008312A400A5014A30B000B1018A0134212C
:101920002E308A014B20A901831623088312A400BC
:10193000A5014A30B000B1018A013421DF308A01AB
:101940004B2043308A014B2020308A014B2020302D
:101950008A014B2020308A014B2020308A014B2005
:101960000230A9007808A400A5014A30B000B101F6
:101970008A01342125308A014B2052308A014B20C4
:1019800048308A014B20FE308A014B20C0308A014A
:101990004B2057308A014B2069308A014B206E3032
:1019A0008A014B2064308A014B2020308A014B2071
:1019B0000330A9004A08A4004B08A5004A30B00033
:1019C000B1018A0134214B308A014B206D308A01EC
:1019D0004B2068308A014B2020308A014B20033095
:1019E000A9003E08A4003F08A5004A30B000B1019C
:1019F0008A013421DF308A014B200A308A01F2212A
:101A00008A150A12E728FE308A014B2001308A012C
:101A10004B202D308A014B200230A900831622086A
:101A20008312A400A5014A30B000B1018A0134211B
:101A30002E308A014B20A901831624088312A400AA
:101A4000A5014A30B000B1018A013421DF308A019A
:101A50004B2043308A014B2020308A014B2020301C
:101A60008A014B2020308A014B2020308A014B20F4
:101A70000230A9007808A400A5014A30B000B101E5
:101A80008A01342125308A014B2052308A014B20B3
:101A900048308A014B20FE308A014B20C0308A0139
:101AA0004B2057308A014B2069308A014B206E3021
:101AB0008A014B2064308A014B2020308A014B2060
:101AC0000330A9004A08A4004B08A5004A30B00022
:101AD000B1018A0134214B308A014B206D308A01DB
:101AE0004B2068308A014B2020308A014B20033084
:101AF000A9003E08A4003F08A5004A30B000B1018B
:101B00008A013421DF308A014B200A308A01F22118
:101B10008A150A12E728FE308A014B2001308A011B
:101B20004B2057308A014B2069308A014B206E30A0
:101B30008A014B2064308A014B2020308A014B20DF
:101B400047308A014B2075308A014B2073308A015F
:101B50004B2074308A014B2020308A014B20033007
:101B6000A9007508A400A5014A30B000B1018A019E
:101B700034214B308A014B206D308A014B20683074
:101B80008A014B20FE308A014B20C0308A014B2055
:101B900057308A014B2069308A014B206E308A0110
:101BA0004B2064308A014B2020308A014B204D307D
:101BB0008A014B2061308A014B2078308A014B200A
:101BC00020308A014B2020308A014B200330A900AD
:101BD0007908A400A5014A30B000B1018A0134217E
:101BE0004B308A014B206D308A014B2068308A01CE
:101BF0004B200A308A01F2218A150A12E728FE30AA
:101C00008A014B2001308A014B2050308A014B2041
:101C100072308A014B2065308A014B2073308A0173
:101C20004B2073308A014B2075308A014B20723073
:101C30008A014B2065308A014B2020308A014B20DD
:101C40000430A9004408A4004508A5004A30B000AB
:101C5000B1018A01342168308A014B2050308A0159
:101C60004B2061308A014B20FE308A014B20C0306E
:101C70008A014B2020308A014B200230A9007708CE
:101C8000A400A5014A30B000B1018A0121213A30F7
:101C90008A014B200230A9007A08A400A5014A302D
:101CA000B000B1018A01212120308A014B2002308D
:101CB000A9007208A400A5014A30B000B1018A0150
:101CC00021212F308A014B200230A9007B08A4007B
:101CD000A5014A30B000B1018A0121212F308A01CB
:101CE0004B200230A900831628088312A400A50106
:101CF0004A30B000B1018A0121210A308A01F22163
:061D00008A150A12E72813
:02400E00753DFE
:00000001FF
